:100000000AC04AC049C048C047C046C045C044C0F5
:1000100044C042C041C011271FBFCFE5D0E0DEBFC2
:0A002000CDBF2ED000C0F894FFCF32
:10002A00A89583FD02C048E001C048E28770842B8E
:10003A0048ED0FB7F894A8954CBF81BF0FBF41B7E1
:10004A00406441BF4AB7417F44604ABF4AB74160F2
:10005A004ABF4FB77894889558ED60E00FB7F89487
:10006A00A8955CBF61B7677F61BF0FBF4FBF4AB733
:06007A004E7F4ABF08950D
:10008000789448ED4CBF41E047BF44E041B944E0BB
:0800900040B986E0CADFFBCF96
:02009800B3CFE4
:02009A001895B7
:00000001FF
